:020000040000FA
:040000000B303A285F
:08000800A000030EA100831209
:1000100005191028831601178312B23081002B288E
:1000200083160113831203140B190310A80DA90DD5
:10003000AA0DAB0DAC0DAC16FF302C02031D2B2806
:10004000FA302B02031D2B2831152A08AF0029088E
:10005000AE002808AD008B100B11210E8300A00EFE
:04006000200E090065
:0C007400203084008001840A6030040207
:10008000031C3C281230B00020228316FF2390006E
:1000900083128316851683120C30851A2C30831632
:1000A000850083128501870107309900003083168F
:1000B00091009F008312C830831681008312313073
:1000C0009000003083168C00831210308B00831652
:1000D00000309B001C141A088312BC00851D9C2252
:1000E0003C1C7A28831610309B001C141A088312BB
:1000F000BD006822831620309B001C141A0883124E
:10010000C1000130C1080319C10081018E018F01B6
:100110000B118B100B108C018B179D203119A02017
:100120000422B30B9B28031085190314B90DF0307A
:1001300039020319962171228D28640032100800BB
:1001400031110130B7008B132030370783169B0025
:100150001C141A088312A4001030370783169B0062
:100160001C141A088312A300A6000230A606003051
:10017000370783169B001C141A088312A200A700DD
:100180000130A7068B17321CCB2822090339A200A5
:10019000A309A409A50924082F02031D90292308F7
:1001A0002E02031D2F2922082D02031D9029013044
:1001B0003702031DE2283C19E1283D18E2283D14CE
:1001C0003E14212202303702031DED283C19EC2891
:1001D000BD18ED28BD143E14282203303702031D3C
:1001E000F8283C19F7283D19F8283D153E142F2210
:1001F00004303702031D03293C190229BD190329C4
:10020000BD153E14362205303702031D0E293C1958
:100210000D293D1A0E293D163E143D2206303702A7
:10022000031D19293C191829BD1A1929BD163E1498
:100230003E2207303702031D24293C1923293D1B88
:1002400024293D173E143F2208303702031D2F2971
:100250003C192E29BD1B2F29BD173E14402226080C
:100260002E02031D902927082D02031D902901301D
:100270003702031D42293C1941293D1C42293D10EA
:100280003E14412202303702031D4D293C194C29EE
:10029000BD1C4D29BD103E14432203303702031DFF
:1002A00058293C1957293D1D58293D113E14452216
:1002B00004303702031D63293C196229BD1D6329DF
:1002C000BD113E14472205303702031D6E293C192B
:1002D0006D293D1E6E293D123E144E220630370216
:1002E000031D79293C197829BD1E7929BD123E14B8
:1002F0004F2207303702031D84293C1983293D1FF3
:1003000084293D133E14502208303702031D8F29E3
:100310003C198E29BD1F8F29BD133E1451229029EF
:10032000B70A0530370203180800A3280130B600C9
:10033000B300B400B500B70004308316851AB700C7
:10034000831285018701B1139D20B30BD3290310BC
:1003500085190314B90DF03039020319FA29B40BC9
:10036000D329013037020319522202303702031910
:1003700056220330370203195A2204303702031978
:100380005E22053037020319622206303702031954
:100390006322073037020319642208303702031939
:1003A00065229630B400311DA4293111321CDD299B
:1003B0002D090339AD00AE09AF092F1CA4298E0108
:1003C0008F010C1CA4290C102E1EA4298B13203085
:1003D0003707BB002F08BA000D2210303707BB00CB
:1003E0002E08BA000D2200303707BB002D08BA00D6
:1003F0000D228B1785018701B70AB6010530370238
:10040000031CA429682208003E1C08003E1010307E
:10041000BB003D08BA000D2208008B133A08831672
:100420001C159A003B089B0055309D00AA309D008A
:100430009C1464009C18192A1C1183128B17080045
:100440000800851440084107D0000F08D1000800BB
:10045000051440084107D2000F08D3000800851694
:1004600040084107D4000F08D500080005164008D1
:100470004107D6000F08D700080008000800080050
:1004800008008510080005100800851208000512F4
:100490008E018F010C104108C00008000800080000
:1004A000080008000508023A850008000508013A1E
:1004B000850008000508203A850008000508103A64
:1004C000850008000800080008000800080008006F
:1004D0003D188514BD1805143D198516BD1905165E
:1004E00008003C1D080050084002031D7C2A5108EA
:1004F0000F02031C7C2A851052084002031D852A26
:1005000053080F02031C852A051054084002031DDE
:100510008E2A55080F02031C8E2A851256084002A7
:10052000031D972A57080F02031C972A05120C1C5B
:1005300008000C10C00A0800B601B301B4013C1C4D
:10054000A42ABC01BC14AB2ABC1CA92ABC013C15C2
:10055000AB2ABC013C143C08B6006400AF2AB02AA8
:10056000B12AB22AB32AB41B8514B41F8510B30B69
:10057000AD2AB40BAD2A0310B60CB608031DAD2A84
:0C0580000030BB003C08BA000D2208004F
:084000000D000300030009009C
:02400E00CC01E3
:10420000010078007A007C007E007B0079007F004E
:104210007D007A0078007E007C00FF00FF00FF0038
:104220000000F200F600FA00FE00F200F600FA00CC
:10423000FE00F200F600FA00FE00FF00FF00FF00A3
:10424000010005000500050005000900090009003E
:1042500009000D000D000D000D00FF00FF00FF0024
:10426000FF00FF00FF00FF00FF00FF00FF00FF0056
:10427000FF00FF00FF00FF00FF00FF00FF00FF0046
:10428000FF00FF00FF00FF00FF00FF00FF00FF0036
:10429000FF00FF00FF00FF00FF00FF00FF00FF0026
:1042A000FF00FF00FF00FF00FF00FF00FF00FF0016
:1042B000FF00FF00FF00FF00FF00FF00FF00FF0006
:1042C000FF00FF00FF00FF00FF00FF00FF00FF00F6
:1042D000FF00FF00FF00FF00FF00FF00FF00FF00E6
:1042E000FF00FF00FF00FF00FF00FF00FF00FF00D6
:1042F000FF00FF00FF00FF00FF00FF00FF00DD00E8
:00000001FF
